:020000040000FA
:0400000000001628BE
:08000800B500030E8301B600F0
:100010000A08B700D80B0E285914C1280B1137084D
:100020008A00360E8300B50E350E090083120313C5
:10003000D9018B018A01850186013330870083163F
:100040000313FF30850084309F00C0308600C43029
:100050008700D321D321D321831203130330BF00A0
:10006000860086160000000000008612D321BF0B18
:1000700031280230860020222830FD210C30FD215D
:100080000630FD213F222A22051975285528051E14
:100090000923851E0E2305194728D91E5028DD2265
:1000A000DD0A5D08033C031D5628DD01D9122A2212
:1000B0001130332200308A005D08820763286928E6
:1000C0006F28132347280030DE00C3222C30332250
:1000D00061280430DE00C322313033226128083029
:1000E000DE00C32220303322612883120313303014
:1000F00087000430F621071200000714831203134F
:1001000081309F00F5211F151F1984281E08D40077
:10011000831603131E0883120313D30083120313E1
:1001200089309F00F5211F151F1994281E08D6003D
:10013000831603131E0883120313D500D90103305D
:100140005602031DA5285914C5281B308700A3217A
:10015000DC21071FA828DC21972103305402031D4E
:10016000B728303087000430F6218712B9281830BC
:100170008700071BB9281014071DC1280C189E21E1
:10018000BC2890018B010C189E211B3087002A226D
:10019000591CCF28253033220E29AA012A172030D6
:1001A0003322A8015708A7000F08A6000E08A500D3
:1001B000051ADE286A2252304E220E294C232030A6
:1001C000C322F6241C30C3222E240830AC22D223B2
:1001D000A8016A22D9140330DC00D9155130592204
:1001E000513059225030592250305922D918FA280A
:1001F0002C3012224F305922D91859154F3059221C
:10020000D9104E305922591D092959112D224E302D
:10021000592231220230122246301222051E632951
:1002200059120330540203192429BA225408A70092
:100230005308A60022230C30C322F6241430C32214
:100240002E240030AC2236290330560203195916E9
:10025000BA225608A7005508A60022231030C32250
:10026000F6241830C3222E240430AC22FC211C308A
:100270003322591E3E293E3012223F29312280303E
:10028000270503194529BA224629D223D911D914A1
:10029000A8016A225030592250305922D9104F30CB
:1002A00059222D224F3059224E3059224E30592298
:1002B000312201301222831203138714CA218312C0
:1002C000031387107528FC2137303322BA225408D3
:1002D000A6005308A5006A224F304E223B3033223D
:1002E000BA225608A6005508A5006A224F304E22B1
:1002F00005195B29282241303322BA225408A7006D
:100300005308A600222396220C30DE00DD22BA22FA
:100310005608A7005508A600222396221030DE00BA
:10032000DD22AF212A2252303322C1215B298E01E6
:100330008F010C1000309000D70108000C10D70F6F
:1003400008005914C1284630D8008101813084004A
:10035000073080000B118B168B1781010800831268
:1003600003131B30B8004E30B9000E30BA00E52937
:10037000831203136730B8008930B9000930BA001E
:10038000E52983120313B330B800C430B900043038
:10039000BA00E529831203135930B8006230B9005E
:1003A0000230BA00E529831203131A30B800063070
:1003B000B9000030BA00E529831203133E30B800BB
:1003C0000030B9000030BA00E529FF30B807031843
:1003D0000301B90703180301BA070318030138041E
:1003E00039043A04031DE52908001F30B800B80B92
:1003F000F729000000000800C030BE003E0E0F3993
:100400008600861600000000000086123E080F39A4
:10041000860086160000000000008612DC2108001D
:100420000F393038BE003E0E0F3910388600861660
:1004300000000000000086123E080F3910388600C8
:10044000861600000000000086128601DC210800EC
:1004500002302B2A0130FD21D3292E30122A3030D0
:10046000122A2030122ABF00BF0307308A003F083B
:100470000027FF39031908001222BF0A372A483023
:10048000FD2107308A001030BF000030C000002777
:100490001222C00A4008BF0B472A08008400000E41
:1004A0001022000810224E300402031908008403B1
:1004B0004F2A8400800E0008D91C622A0F390319C4
:1004C0000800D910D91D102ADC0803192F2ADC03D3
:1004D000102208002030C200CE01CF01D001D1018E
:1004E000D201A50DA60DA70DA80DCE0DCF0DD00DD7
:1004F000D10DD20DC20B7D2A08000530C0004E3050
:100500008400832A840A8722C00B822A712A03303E
:100510000007C100C119800030300007C100C11BB5
:1005200080000800BB002830BC009D2A2830BC0099
:100530002F309C2ABC002830BB000430BF003C0890
:1005400084000008BD003B0884003D088000BB0318
:10055000BC03BF0B9F2A0800C322B1224C232E24C8
:100560000800463092222F309A2246309722080007
:100570002F30BB2A283084000430BF008001840360
:10058000BF0BBE2A0800DA002F3084000430BF0001
:10059000D122831203138000DA0A8403BF0BC82A16
:1005A00008005A08831203178D00831603178C1353
:1005B0000C14831203170C0808005E08DA002F30B1
:1005C00084000430BF000008DB00ED228312031317
:1005D000DA0A8403BF0BE32A0800831603178C187A
:1005E000EF2A831203135A08831203178D00831214
:1005F00003135B08831203178C00831603178C13F5
:100600000C1555308D00AA308D008C1400000C1193
:100610000800D916AC0A0319AD0A132BD916AC0879
:100620000319AD03AC032F309A226A22FC214F300C
:1006300059222D224F3059224E3059224E30592204
:10064000CA2108008E30A8002708A900A71F2D2B5B
:10065000A609A709A60A0319A70AB3012708031DBB
:10066000372B2608A7000319472BA601B31533081B
:10067000A802031D031CEA2C0310A71B442BA60D84
:10068000A70DA80B3D2BEA2CA91FA7130034A70127
:10069000A601A501A80100349630A800A901A71F52
:1006A0005A2BA509A609A709A50A0319A60A031921
:1006B000A70AA917B3012708031D6F2B2608A70057
:1006C0002508A600A501B3152708031D6F2B2608D2
:1006D000A700A601B311331627080319472B3308C7
:1006E000A802031D031CEA2C0310A71B7D2BA50DDC
:1006F000A60DA70DA80B752BEA2C2A1B261C442B34
:10070000A51F442BA60A0319A70A031D442BA70CF7
:10071000A60CA80A0319742C442B280803190034CA
:100720002708A900A7178E30A802A81FC72BA80961
:10073000A80A08302802031CAD2BA800A60D270824
:10074000A600A70108302802031CAD2BA800A60DA7
:10075000A6012808031D0310B52B28080319B52B83
:100760000310A70CA60CA80BB02B2A1B261CBF2B12
:10077000031CBF2BA60A0319A70AA71BC72BA91F77
:100780000034A609A709A60A0319A70A00342A14E7
:10079000AA1FFF34A701A91FFF30A700A600A90DBB
:1007A000A70CFF34A5012808031900342708A90065
:1007B000A7179630A802A81F222CA809A80A08305B
:1007C0002802031CFE2BA800A50D2608A50027085B
:1007D000A600A70108302802031CFE2BA800A50DC7
:1007E0002608A500A60108302802031CFE2BA8003D
:1007F000A50DA5012808031D0310072C28080319BF
:10080000072C0310A70CA60CA50CA80B012C2A1B67
:10081000251C132C031C132CA50A0319A60A031963
:10082000A70AA71B222CA91F0034A709A609A509FE
:10083000A50A0319A60A0319A70A0034A701A601ED
:10084000A50100342A14AA1FFF34A701A91FFF30F5
:10085000A700A600A500A90DA70CFF342808031DBA
:100860002F080319472B27082E06A9002F08A807D1
:100870007E30031C3F2CA8020318742C422CA802C3
:10088000031CEA2C2708A5002608A400A517AE170C
:100890000310A701A6011030B300241C552C2D080D
:1008A000A6072E0803182E0FA707A70CA60CA50C49
:1008B000A40C0310B30B4D2CA71B622CA50DA60D89
:1008C000A70DA8032A1B261C712CA51F712CA60A94
:1008D0000319A70A031D712CA70CA60CA80A03195B
:1008E000742CA91FA7130034AA14AA1FFF34FF30C9
:1008F000A800A700A600A90DA70CFF342F08031914
:10090000F42C28080319472B27082E06A900A7173F
:10091000AE17B3012708A5002608A4002D08A402DD
:100920002E08031C2E0FA502A501A401031C9E2C5A
:100930000310A70CA60CA50C0130B3002F08A802C9
:10094000031CA82C7E303307A8070318742CAD2C89
:100950007E303307A807031CEA2C1030B200A40D28
:10096000A50DA60DA70DB30D2D08A6022E08031C7C
:100970002E0FA7022E0DB304331CC02C2414C72C39
:100980002D08A6072E0803182E0AA7072410B20B5D
:10099000AF2C2A1B241CE32C0310A60DA70DB30DAE
:1009A0002D08A6022E08031C2E0FA7022E0D3304BD
:1009B0000139A4070318A50A031DE32CA50CA40CF8
:1009C000A80A0319742CA91FA5132508A700240839
:1009D000A60000342A15AA1FFF340130A800A70181
:1009E000A601A90DA70CFF34AA15FF348030AE066E
:1009F00027082E06B300A501AC0128082F02031C0E
:100A0000132D2F08A3002808AF002308A8002E08E4
:100A1000A3002708AE002308A7002D08A30026087E
:100A2000AD002308A6002F08031900342708A900E9
:100A3000A717AE172F082802AF000319392D083069
:100A40002F02031C302DAF002D08AC002E08AD0086
:100A5000AE0108302F02031C302D2908A7000034F6
:100A60002F080319392D0310AE0CAD0CAC0CAF0BD5
:100A7000332DB31F432DAC09AD09AE09AC0A0319E0
:100A8000AD0A0319AE0A2C08A5072D0803182D0F6F
:100A9000A6072E0803182E0FA707B31B572D031CFC
:100AA0007D2BA70CA60CA50CA80F7D2B742C03186E
:100AB0005A2BA509A609A709A50A0319A60A03190D
:080AC000A70A8030A9062D2BC6
:100E0000820700340E341134113411340A341B3487
:100E10000034003400341234123412341E341134CD
:100E2000103443346F346534663466342E342034E1
:100E300066346F34723400344534533452340034E1
:100E4000203443347834203400344334783420342C
:100E50002D342D342D3400342034313420340134F9
:100E6000003420343134303420340134003431340F
:100E700001343D34003420343134303401343D34D5
:100E800000345534303420342D342D342D343E3458
:100E9000203445344534503452344F344D342034AA
:100EA00020340034493474342034693473342034A9
:0E0EB000723465346134643479342134003492
:02400E00323F3F
:10420000000000000300E800000000000300E800D8
:10421000000000000300E800850016000000000018
:1042200081006000000000007500400030000C00BC
:104230007800740089008D0074002E00C3003E00D9
:084240008000400000000000B6
:00000001FF
